:020000040000FA
:030000000200916A
:03001B0002025C82
:100073000202C200000080FBE4900281780A790248
:100083008002F0A3D8FCD9FA12045112007675D07D
:100093000075813F750A81750B0202007BCAC0E0BF
:1000A300E6F0A308DAFAD0E0FA22250A10AF08F541
:1000B3000A400C150B8008F50A4002150BD2AF223B
:1000C30000C0D0250A10AF08F50A500C050B8008B4
:1000D300F50A5002050BD2AFD0D022250AF58210C3
:1000E300AF08F50A400C150B8008F50A4002150B02
:1000F300D2AF850B8322250AF582E4350BF58322E3
:10010300250AFAE4350BFB22E473250AC582C0E015
:10011300E50B34FFC583C0E0E50AC3958224F910DB
:10012300AF0885830B85820A800885830B85820A45
:10013300D2AFCEF0A3E520F0A37808E608F0A3DE63
:10014300FAEFF0A3E58124FBF8E608F0A3E608F054
:10015300A30808E608F0A3E608F0A315811581D0EB
:10016300E0FED0E0F815811581E8C0E0EEC0E022A2
:10017300850B83850A82E0A3FEE0A3F5207808E0DF
:10018300A3F608DFFAE0A3FFE0A3C0E0E0A3C0E02A
:10019300E0A3C0E0E0A3C0E010AF0885820A858336
:1001A3000B800885820A85830BD2AFD083D082224D
:1001B30074028000C0E0F4041200DED0E01200A05C
:1001C30022C082C083900301E0FAF8A3E0C39A40FF
:1001D30008E0C398F895E0800F7480C398FA95E01F
:1001E300FBE0F8EA28F8E43BF97A00A3E0FC6016A8
:1001F300A3E0FBE595C39BFBC39C9003035005E081
:10020300C39B8001E4F0E595A3F0C3E8947FE994F0
:100213000040047A018019C3E89430E99400400453
:100223007A02800CE8496008900303E070027A04C4
:10023300900387E06006E4F0EAD2E4FAEA6015A3EB
:10024300E0F8A3E0F988828983E582458360057934
:100253000112010BD083D08222C0E0C0D0E8C0E0FD
:10026300E9C0E0EAC0E0C082C083A2AFE433FAD2BF
:10027300AFA8F9E8C0E0900302E0F8748128F582A2
:10028300E43402F583D0E0F0900301E0F8A3E068E2
:100293007006E595900304F0900302E004F0C39424
:1002A300804002E4F0A3E4F0EAA2E092AFD083D06E
:1002B30082D0E0FAD0E0F9D0E0F8D0D0D0E032C07C
:1002C300E0C0D0E8C0E0E9C0E0EAC0E0C082C0839B
:1002D300A2AFE433FAD2AF900385E0F8A3E06870ED
:1002E30008539AF7A374018022C2EA900385E0F8C9
:1002F300740128F0740528F582E43403F583E0F5EE
:10030300F9900385E0C394804002E4F0809A53FFA0
:100313003F43FF4043F10243F4C053F23F75F8807B
:1003230075FB8022C082C083E9FC74016C60030208
:1003330003BDEA241BF582E43BF583E0F8A3E0F96F
:10034300900388E8F0A3E9F08A828B83A3E0F87432
:100353000368600A740468600575FA3B800375FAE4
:10036300D8E0601F14601714600F14600C24FE6043
:100373001714601914601B801E75FC0A801C75FC21
:1003830009801775FC08801275FC07800D75FC0643
:10039300800875FC05800375FC0B8A828B83A3A3FD
:1003A300E0600D75FB4243F430C29543FE208003A9
:1003B30075FB02D2ABD2EA75F8C07900020257741A
:1003C300F812010D8908EAF8EBF9740165087A005F
:1003D3007B007041802E74812EF582E43402F58314
:1003E300E088828983F0900301E004F088828983A6
:1003F300A3A882A983C394804005900301E4F00A73
:10040300EA70010B900301E0FEA3E06E6007C3EA0C
:100413009CEB9D40C17F010201730201C474F7127A
:10042300010D74FF1200AD7C017D00AA0AAB0B1213
:1004330003C28B09EA4509600B850A82850B83E0B9
:10044300906185F074011200C37F0202017374E3AB
:100453001200AD53BEFBE59DA2E650FAE5C65480FB
:100463004449F5C6E59E547F644970F853C680E558
:100473009E547F70FA43BE049062707408F043F494
:100483000875CB1275CC1475CD9F43FE041203116E
:1004930075081D75090078081201B37C007D00748E
:1004A300021201031204CE74021200C3740112007B
:1004B300F9E4F0741B1200F97420F0A37404F079CA
:1004C30001120327D2AF12041D80FBC082C08385B3
:1004D3000A82850B83E0F8A3E0F9E84960128A8277
:1004E3008B83ECF0A3E824FF18E934FFF94870F29A
:0504F300D083D082223D
:040000050000009166
:00000001FF
